:100C7F007E306D79335B5F707F7B771F4E3D4F0109
:100C2F00EF4E60147D737C00ED1D70011CED4C7058
:080C3F00F7EF1F70EB1E80E8C7
:010C4700228A
:090CDE007F087808E4F608DFFC49
:010CE70022EA
:0A0CE800E4F50CF50DF50EF50F22F2
:0C0CBA00C2957FF47E01120C2FD295220F
:0C0CC600C2957F327E00120C2FD29522C6
:040A6600AB05AA042E
:100A6A007D01EF339291EF25E0FFD293C2930DBD42
:100A7A0009F07D01EB339291EB25E0FBEA33FAD2E0
:0B0A8A0093C2930DBD09EDD292C29201
:010A9500223E
:100B2100C293C292E4FDFC7F0F120A667D017F0C25
:100B3100120A66E4FD7F09120A667D0F7F0A120A16
:080B4100667D077F0B020A66C6
:1008BA00120B21E508FD7C007F01120A66E509FD9D
:1008CA007F02120A66E50AFD7F03120A66E50BFD3E
:1008DA007F04120A66E50CFD7F05120A66E50DFD26
:1008EA007F06120A66E50EFD7F07120A66E50FFD0E
:0508FA007F08020A6600
:090D0600000000000000000022C2
:050D0F00D297020D0661
:050D1400C297020D066C
:060C4800120CF2120D0671
:0E0C4E00D296D297C296120D06C297D2962267
:0A0CF200C296D297120D06D2962288
:070A3500120C4E7FD07E0081
:100A3C007D01EF339204A2049296EF25E0FFEE3392
:100A4C00FE120D0F120D140DBD09E7D296120D0FEB
:090A5C00A2969204120D14A204EA
:010A6500226E
:100A9600E4FF7E01120D0FA2969204EF25E0FFA25D
:100AA60004E4334207120D140EBE09E8D296120D65
:0F0AB6000FA2969204120D14A204B350027FFFF8
:010AC500220E
:100B7100E4FF7E01120D0FA2969204EF25E0FFA281
:100B810004E4334207120D140EBE09E8C296120D99
:060B91000F120D14D296B4
:010B9700223B
:0A0CFC0053107F5312BF5317EC2270
:100BDB00120A35E4FFFE120A3CE4FC74102CF8E612
:0D0BEB00FF7E00120A3C0CBC08F1020CF267
:100AF500120A35E4FFFE120A3C120C487FD17E0033
:100B0500120A3CE4FD120B71AC0774102DF8A60413
:0C0B15000DBD07F1120A968F17020CF2BA
:1009FF00120A357F087E00120A3CE4FC74502CF872
:100A0F00E6FF7E00120A3C0CBC08F1E4FC74232CB8
:100A1F00F8E6FF7E00120A3C0CBC08F1AF2B7E00FB
:060A2F00120A3C020CF269
:1009C500120A357F087E00120A3C120C487FD17E40
:1009D50000120A3CE4FD120B7174502DF8A6070DA8
:1009E500BD08F3E4FD120B7174232DF8A6070DBDA8
:0A09F50008F3120A968F2B020CF291
:060CAD0054F0C4540FFFD7
:070CB300EF900C7F93FF227C
:0C0BBB00AF0A120BC7EFC454F0FDAF0BE3
:100BC700E4FEEE900C7F93B50703AF06220EBE102E
:030BD700F17FFFAC
:010BDA0022F8
:1008FF00E53C120CAD8F08E53C540FFF120CB38F83
:10090F0009E53D120CAD8F0AE53D540FFF120CB3F4
:10091F008F0BE53E120CAD8F0CE53E540FFF120C02
:10092F00B38F0DE53F120CAD8F0EE53F540FFF1245
:05093F000CB38F0F2234
:10094400AF08120BC7EFC454F0FDAF09120BC7EF89
:100954004DF53C120BBBEF4DF53DAF0C120BC7EF41
:10096400C454F0FDAF0D120BC7EF4DF53EAF0E12A0
:100974000BC7EFC454F0FDAF0F120BC7EF4DF53F9B
:010984002250
:1007CA00E4FE74082EF8E6547FF60EBE07F4EF1422
:1007DA00B40700503E9007ED75F003A4C58325F0D9
:1007EA00C5837302080202080602080A02080E02FA
:1007FA00081202081602081A4308802243098022B6
:10080A00430A8022430B8022430C8022430D80221C
:03081A00430E800A
:01081D0022B8
:0F0C8F0085123C85113D85143E85153F0208FFF7
:100C6F00120944853C12853D11853E14853F15229E
:100BF800E4FE2090077F14DFFE0E80F630900B7F16
:0C0C080014DFFE0EBEFFF5AF0622AF06A3
:010C140022BD
:10010E007B107840E4F608DBFC7B10120BF8120B28
:10011E00F8120BF8120BF8120BF8AA07EAF460317A
:10012E00854140854241854342854443854544850A
:10013E004645854746854847854948854A49854B02
:10014E004A854C4B854D4C854E4D854F4E8A4F8082
:10015E00C679FFE4FB74402BF8E6FFC3995002A961
:10016E00070BBB10F0E925E02404F56B74FC29F9AC
:10017E00E4FB74402BF8E6FAC3994006EAD3956B7C
:10018E0040037F00220BBB10E9120CC67558167582
:10019E0059A8C2007F327E00120C2F200117E4FBFB
:1001AE0074402BF8E6FF742C2BF8A6070BBB10F04F
:1001BE00D2017F0222E4FB74402BF8E6FA742C2B5A
:1001CE00F8E6FF24FCF9EF2404F56BEAC399400628
:0F01DE00EAD3956B40037F01220BBB10DA7F023F
:0101ED0022EF
:10081E007F057E00120C2F20900302010E30B103D3
:10082E0020B02120031B20B105756A018003756A73
:10083E0002120CC6D2037558167559A8C200AF6ABB
:10084E00227F0022C203D3E5599400E5589400405C
:10085E0010E559155970021558E55945587002D2D0
:03086E00007F0008
:010871002264
:040561007D097F038E
:040565008F648D65AD
:10056900E4F567F56874082FF8E6FF120BC78F6684
:1005790012081EBF020E0566E566D395654048E47C
:10058900F5668043BF0111AF66120CB37408256488
:10059900F8A6071208BAC3220568E568700205675C
:1005A900641945677021F567F568B20430040EAF28
:1005B90066120CB374082564F8A607800774082529
:0B05C90064F8E4F61208BA3000A6D374
:0105D4002204
:040471008F658D66A0
:10047500E4F568F56974082FF8E6FF120BC78F6776
:1004850012081EBF0218E567B40F05E4F567800280
:100495000567E567D39566404875670F8043BF01DB
:1004A50011AF67120CB374082565F8A6071208BAD0
:1004B500C3220569E56970020568641945687021FC
:1004C500F568F569B20430040EAF67120CB3740811
:1004D5002565F8A607800774082565F8E4F612086F
:0504E500BA30009CD3B9
:0104EA0022EF
:10076900E4F565F566AF0B120BC78F6412081EBF5F
:10077900020E0564E564D394074041756401803C29
:10078900BF010CAF64120CB38F0B1208BAC3220558
:1007990066E5667002056564194565701FF565F5BE
:1007A90066B20430040BAF64120CB38F0BAF6480D4
:1007B90005E4F50B7FFF1207CA1208BA3000ADD362
:0107C900220D
:10098500750A08750B08E521700775080F75097656
:1009950022E521B4010775084E75090E22E521C32C
:1009A5009406500D75087775090EE521900C7E802B
:1009B5000B75085B75093DE521900C7A93F50B22C3
:10087200E4F564F56512081EBF020B0521E521D3DC
:100882009409402FD322BF01081209851208BAC366
:10089200220565E56570020564641945647014F506
:1008A20064F565B2043004051209858003120CDE7A
:0708B2001208BA3000BFD3A9
:0108B900221C
:10037100900C7FE493F508F509F50AF50B7D05E48A
:10038100FF120565406D7D097F0112056540647DA1
:10039100057F02120565405B1205614056AF0812E8
:1003A1000BC7EF4430F55CAF09120BC7EF4430F5D2
:1003B1005DE4F55EFB7A00795C1201EE8F5AAF0ABB
:1003C100120BC7EF4430F55CAF0B120BC7EF443093
:1003D100F55DE4F55EFB7A00795C1201EE8F5B124C
:1003E1000AF5AB107F147E00120C2F120AF5E510EE
:0303F1006B60F14D
:0103F40022E6
:1002CC00120C8F7D02E4FF12056550030203707D52
:1002DC00097F0112056550030203707D057F021230
:1002EC000565500302037012056140787D037F049D
:1002FC00120565406F7D097F0512056540667D011D
:10030C007F06120565405D7D097F07120565405427
:10031C00120C6F75083E75093D750A08AF13120C67
:10032C00B38F0B120769403CAF0B120BC78F1375C1
:10033C00083B750908E516120CAD8F0AE516540F2B
:10034C00FF120CB38F0B7D097F021205654015124D
:10035C0005614010120BBBEF4DF516E4F510120CB5
:05036C00FC120BDB2276
:0206A200AE07A1
:1006A400EE1425E0F5642423F8E6F53C742425646F
:1006B400F8E6F53D1208FF750C77750D0E750E08FA
:1006C400AF06120CB38F0F7D02E4FF1204714032A7
:1006D4007D097F0112047140297D057F0212047196
:1006E40040207D097F0312047140171209447423CA
:1006F4002564F8A63C74242564F8A63D752B0112E4
:0207040009FFEB
:0107060022D0
:02070700AE073B
:10070900EE1425E0F5642450F8E6F53C74512564AF
:10071900F8E6F53D1208FF750C5B750D3D750E0881
:10072900AF06120CB38F0F7D03E4FF120471402F43
:100739007D097F0112047140267D017F0212047137
:10074900401D7D097F03120471401412094474503D
:0F0759002564F8A63C74512564F8A63D1209FFEB
:01076800226E
:10063C00120CDEE4F521120872405AE521B40A00CE
:10064C0050F4900655F828287302067302067602B9
:10065C00067B02067F02068302068702068E0206CE
:10066C009202069602069A0203711202CC80C77F90
:10067C0001800A7F0280067F0380027F041206A29B
:10068C0080B47F01800A7F0280067F0380027F0492
:06069C0012070780A122F5
:100C15007F647E00120C2F120CDE1208BA120CBA79
:0A0C25001209C57F907E01020C2F1A
:1005D50030B0FDE4F56574502565F876FF0565E5F1
:1005E50065B408F2E4F56574232565F876FF0565BD
:1005F500E565B408F2E4F52B1209FF756401B294C0
:10060500E4F56574082565F8A6640565E565B4082F
:10061500F21208BA12081EEF60FABF010DE564C3B5
:1006250013F56470D975648080D4E56425E0F564BC
:0706350070CC75640180C761
:100AC600120CDE20B128120AF585103D85163F125C
:100AD60008FFE4F508F509750C3B750D08AF131210
:0F0AE60007CA1208BA7F647E00120C2F80D52237
:1003F500E55A7007E55B7003300270AE5AEE75F092
:100405000A84AFF0120CB38F0DEE75F00A84FE75F9
:10041500F00A84AFF0120CB38F0CAE5BEE75F00AE8
:1004250084AFF0120CB38F0FEE75F00A84FE75F0F1
:100435000A84AFF0120CB38F0E900C7FE493B50CC9
:1004450003E4F50CE55AD394005006E55B940040AF
:100455001AE55B7007155A755B3B8002155BE55A1B
:0B0465007009E55B7005D20275220AE9
:010470002269
:100B4900E52B64017021E510701D7F01EF1425E08C
:100B5900FE2423F8E6B5120B74242EF8E6B511032A
:070B690075221E0FBF05E518
:010B70002262
:100B98007D01ED1425E0FF2450F8E6B514107451DA
:100BA8002FF8E6B51508120CE8AF131207CA0DBDE9
:020BB80005E056
:010BBA002218
:10000300E4F55FF5607561FF120C1520B00312056E
:10001300D5E560455F60030200A8F55F75600512D2
:100023000AF5E5106561604C851061C201120C8F01
:10003300900C7FE493FFB50803E4F508E50CB507DE
:1000430003E4F50CE522D394004004C29515221273
:1000530003F5E5227002C202120B49E4F562430F75
:1000630080AF131207CAE52BB40104C2948002D2F5
:10007300941208BA0562E562D3940C4030530F7FA3
:10008300D295E55AD39400500CE55B94005006E5F5
:100093002294004008120CE8AF131207CA120B98FF
:1000A3001208BA8008E56015607002155F12081E19
:1000B3008F63E563600DE522D394004006E4F522E7
:1000C300020014E563B4020912063C7561FF0200E5
:1000D30014E56364016003020014E55A600302003F
:1000E30014E55B6003020014E52B7005752B01809A
:1000F30003E4F52BE52BB40104C2948002D29412DD
:0B01030009FF120AC67561FF0200141C
:03000000020CD21D
:0C0CD200787FE4F6D8FD75816B0200030A
:1001EE008B648A658966AB64AA65A9661204EBFF07
:1001FE00120C5C500D74012566F566E43565F565E7
:10020E0080E4D204AB64AA65A9661204EBFF642BEA
:10021E006004EFB42D1BAB640566E566AA6570023B
:10022E00056514F91204EB642D6003D38001C392AB
:10023E0004E4F56AF569F568F567AB64AA65A96625
:10024E001204EBFF120C9E505CE47F0AFEFDFCAB29
:10025E006AAA69A968A867120504C8ECC8EDC0E0CF
:10026E00EEC0E0EFC0E0AB64AA65A9661204EBFF36
:10027E003395E0FEEF24D0FFEE34FFFEE4FCFDD01C
:10028E00E0FBD0E0FAD0E0F9EB2FF56AEA3EF56933
:10029E00ED39F568EC38F56774012566F566E435D9
:1002AE0065F565809530040AAF6AAE69AD68AC67D6
:0E02BE00800BAF6AAE69AD68AC6712055322C3
:1004EB00BB010689828A83E0225002E722BBFE020F
:0904FB00E32289828A83E4932242
:10050400E88FF0A4CC8BF0A42CFCE98EF0A42CFC96
:100514008AF0EDA42CFCEA8EF0A4CDA8F08BF0A414
:100524002DCC3825F0FDE98FF0A42CCD35F0FCEB73
:100534008EF0A4FEA9F0EB8FF0A4CFC5F02ECD3938
:0F054400FEE43CFCEAA42DCE35F0FDE43CFC22A5
:0E055300C3E49FFFE49EFEE49DFDE49CFC22B9
:0F0C9E00EFC394304007EF943A50028001C32215
:100C5C00EFC394094005EF940E4003BF2003D380EB
:030C6C0001C3229F
:00000001FF
